:100000001AC034C033C032C015C230C02FC02EC099
:100010002DC02CC096C12AC029C028C027C00037D7
:10002000003800360101010101010102040810201D
:1000300001030000000011241FBECFE5D2E0DEBFA7
:10004000CDBF10E0A0E6B0E0EAE1F7E002C0059025
:100050000D92A236B107D9F710E0A2E6B0E001C0D8
:100060001D92A337B107E1F7D2D155C3C9CFBB9ACF
:10007000B89AB39A0895EF92FF920F931F93CF937C
:10008000DF939C01660F771F660F771F88EE93E062
:10009000F9D2EB017B010027F7FC0095102F84E0DB
:1000A000B901A801970145D0C801B70133D284E056
:1000B00024D184E06AE570E0A80197013AD0CE012E
:1000C00064E070E0DFD2882777FD8095982F22D2F8
:1000D00084E013D1DF91CF911F910F91FF90EF90AA
:1000E0000895CF93DF93809162008F5F80936200C9
:1000F000843611F4109262008091620080FD02C08B
:10010000B39AB09ACFE5D0E0CE0162E070E0B3DF01
:100110002196C936D105C1F7C9E6D0E0CE0162E02B
:1001200070E0A9DF2197CF35D105C1F7DF91CF91DD
:100130000895BF92CF92DF92EF92FF920F931F9399
:10014000CF93DF93082FEB0169017A018091600062
:100150008F3F09F040C013BE1ABC12BE19BC18BCB8
:1001600089B7857E89BF88B78A6188BF8AB58C7F49
:1001700082608ABD83B7877F83BF023080F410928C
:1001800068001092670010926900002321F48AB57C
:100190008F7380641AC08AB58F7C806116C0802FEF
:1001A00090E0FC01EC5DFF4FE491F0E0E05EFF4F7A
:1001B000E491E093670010926800865D9F4FFC0118
:1001C0008491809369008AB58F708ABD802F61E029
:1001D000EDD100936000B0906000B01609F083C0CC
:1001E00083B7887F83BF12BE209709F476C0C230E0
:1001F000D10590F0C830D10588F0CF31D10598F005
:10020000C43FD105A8F0F7E0CE39DF07B0F402E033
:1002100010E028E030E015C0C2E0D0E005E010E0DA
:1002200020E034E00EC004E010E020E031E009C03E
:1002300003E010E020E430E004C001E010E021E041
:1002400030E0BE0180E090E040E050E002D29B014F
:10025000AC01220F331F441F551F60E874E88EE184
:1002600090E023D22F5F3F4F4F4F5F4F56954795FA
:1002700037952795215029BDC114D104E104F1041B
:10028000B1F0CC0FDD1FBE0180E090E0A701960128
:10029000E0D128EE33E040E050E007D22093630045
:1002A0003093640040936500509366000EC08FEF5A
:1002B0009FEFDC018093630090936400A09365003E
:1002C000B09366008B2D823018F089B7806189BFAA
:1002D00083B7887F802B83BF06C089B7857E89BF9F
:1002E000802F60E084D1DF91CF911F910F91FF901B
:1002F000EF90DF90CF90BF900895909160009F3F66
:10030000F9F0981711F08F3FD9F489B7857E89BF2E
:1003100083B7887F83BF23D1E0916700F0916800A5
:10032000309739F09081809169008095892380838E
:1003300004C08091600060E05AD18FEF809360002C
:1003400008951F920F920FB60F9211242F933F938F
:100350004F935F936F937F938F939F93AF93BF93CD
:10036000EF93FF938091630090916400A0916500EA
:10037000B09166000097A105B105B1F180916300CD
:1003800090916400A0916500B0916600181619065E
:100390001A061B06FCF48091630090916400A09102
:1003A0006500B09166000197A109B10980936300CF
:1003B00090936400A0936500B09366008091630001
:1003C00090916400A0916500B09166000097A1052E
:1003D000B10551F0E0916700F09168008081909143
:1003E00069008927808302C08FEF87DFFF91EF913B
:1003F000BF91AF919F918F917F916F915F914F913D
:100400003F912F910F900FBE0F901F901895B4D071
:100410002EDE67DEFECF83B7887F83BF8AB58C7FF1
:1004200081608ABD83B7877F83BF83B7887F8260FF
:1004300083BF08951F920F920FB60F9211242F932E
:100440003F938F939F93AF93BF9380916E00909152
:100450006F00A0917000B091710030917200232F55
:100460002A5F2D3728F02D570396A11DB11D03C01B
:100470000296A11DB11D2093720080936E0090938F
:100480006F00A0937000B093710080916A0090910A
:100490006B00A0916C00B0916D000196A11DB11D83
:1004A00080936A0090936B00A0936C00B0936D00F2
:1004B000BF91AF919F918F913F912F910F900FBE60
:1004C0000F901F9018959FB7F89420916A00309173
:1004D0006B0040916C0050916D008FB508B602FE24
:1004E00006C08F3F21F02F5F3F4F4F4F5F4F9FBFA1
:1004F000542F432F322F2227280F311D411D511D0C
:1005000083E0220F331F441F551F8A95D1F7B9018D
:10051000CA010895EF92FF920F931F93CF93DF9339
:100520007B018C01D0DFEB010EC0CDDF6C1B7D0B9E
:1005300083E0683E780738F00894E108F108010983
:100540001109C851DC4FE114F1040105110569F7E7
:10055000DF91CF911F910F91FF90EF90089513BEFF
:100560001ABC12BE19BC18BC89B7857E89BF88B772
:100570008A6188BF50DF0895789480B7806880BF13
:1005800080B7806480BF8CB580648CBD8FEF8DBDDB
:1005900080B7807F846080BF89B7846089BF3BDF7C
:1005A00086B1887F836086B9379A089590E0FC0110
:1005B000E65DFF4F2491FC01EC5DFF4FE491EE23DB
:1005C000A9F0F0E0E25EFF4FA491B0E0662341F4B1
:1005D0009FB7F8948C91209582238C939FBF0895A8
:1005E0009FB7F8948C91822B8C939FBF0895282FEE
:1005F00030E0F901E65DFF4F9491F901EC5DFF4FAA
:10060000E491EE2329F1882319F48AB58F7304C08D
:10061000813021F48AB58F7C8ABD05C0843019F4FD
:100620008CB58F7C8CBDF0E0E05EFF4FA491B0E014
:10063000662341F42FB7F8948C91909589238C937D
:100640002FBF08952FB7F8948C91892B8C932FBFCF
:100650000895FF27EE27BB27AA2760FF04C0A20F3B
:10066000B31FE41FF51F220F331F441F551F96951C
:1006700087957795679589F70097760771F7CF018A
:10068000BD01089597FB092E07260AD077FD04D0F7
:100690002ED006D000201AF4709561957F4F0895F2
:1006A000F6F7909581959F4F0895A1E21A2EAA1B07
:1006B000BB1BFD010DC0AA1FBB1FEE1FFF1FA21712
:1006C000B307E407F50720F0A21BB30BE40BF50B0F
:1006D000661F771F881F991F1A9469F76095709598
:1006E000809590959B01AC01BD01CF010895AA1B97
:1006F000BB1B51E107C0AA1FBB1FA617B70710F00D
:10070000A61BB70B881F991F5A95A9F7809590953E
:0A071000BC01CD010895F894FFCF5D
:02071A00FF00DE
:00000001FF
